:020000003428A2
:10000800803120007F08F1000B1D31280B11F91CED
:100018001D287D3095000130F702031D3128760830
:10002800F0007008F7000130A602031D312879148A
:100038003128063095000130A7022708031D2C2817
:100048007D30F0007008A7000430F0007008F80058
:100058007808031931280130F8027108FF000900F7
:100068003528F901F601F701F801A501A6012000DC
:10007800482FA02DA52DA92D362E362E362E362EFC
:10008800362EAA2DAE2DB22DB62DBA2DBE2DC22DCF
:10009800C62DCA2DCE2DD22DD62DDA2DDE2DE22D50
:1000A800E62DEA2DEE2DF22DF62DFA2DFE2D022E3F
:1000B800062E0A2E0E2E122E162E1A2E1E2E222E28
:1000C800262E2A2E2E2E322E9B2E9D2E9F2EA12E90
:1000D800A32EA52EA72EA92EAB2EAD2EAF2EB12E58
:1000E800B32EB52EB72EB92EBB2EBD2EBF2EC12EC8
:1000F800C32EC52EC72ECB2ECD2ECF2ED12ED32E2E
:06010800D52ED72ED92EE2
:100200002634A6348634A8346A346034AA348A3456
:10021000A83486348334A33460348634A8348A34D2
:10022000AD348D34AD348F34AF348D34AD34683467
:100230006034A0348D34AA348D34AD348D34AD3473
:100240008E34A0348E34AE3491348F34AF346A346B
:100250008034A8348A34AD348D34AD348A34AA3431
:100260008834A8348634A634003426348234823468
:10027000A23447344E348B34AA34893453346E3428
:100280008B34AA34893453346E348B34AA348B348F
:10029000493482348234A23447344E348B34AA3405
:1002A000893453346E348B34AA34893453346E34E5
:1002B0008B34AA348B3449346234A23444348E34BF
:1002C0008B348A3489348734A7348934AA34693426
:1002D000003430346D348D34AB34AD34AF34AD34A0
:1002E000AB34AA348D34AD34AA346D348D34AB3490
:1002F000AD34AA34A834A534A6344834A834A6347E
:10030000A534A334A534A634A834AA346834683498
:10031000A834AA34AB34AA34A834A634A534A33400
:10032000A534A33481348134A134A3348534863494
:1003300063344834003420349434A034B434B134B9
:10034000A034943480349634803492348034A03491
:100350009434A034B434B134A034943480348F3421
:10036000803480349434A034B434B134A034943420
:1003700080349634803492348034A034943494346D
:10038000803498349834803499349934003440342B
:1003900094349134A034B134B134B434B6348F349D
:1003A000A034AF34B13492349934B934B934B83458
:1003B000B434B634B434B2349134A034B434B63432
:1003C0009634B634BB34B934B834B834B934B634EE
:1003D0009434A034AD34AF34B134B634B63494343C
:1003E00000343034B134B634B134B834B134B43408
:1003F000B634B134B934B134BB34B134B834B934AF
:10040000B134B834B134B634B134B834B134B434AE
:10041000B634B134B934B134BB34B134B834B9348E
:10042000B134B834B134B634B134B834B134B4348E
:100430009634003437349934993499349934993452
:10044000963491349434943492349234A034983461
:10045000983498349834983494348F349134A03448
:100460009134913491349134913496349934983450
:10047000983496349B349B34963499349934983418
:100480009834003430348F349434B434B6349834DF
:1004900094349B349B349834B8349934BB34B93495
:1004A000B834B9349B34B634B434B634B834963432
:1004B0008F349434B434B634983494349B349B34AD
:1004C0009834B834B934BB34B834B9349634B4340D
:1004D000943400342034B934A034B234B434B63453
:1004E000B6349934B234A034B234A034BB34A0341E
:1004F000B634B934BB34BD349E34B234A034B234D3
:10050000A0349634B934B634B634B4349634B634F0
:10051000B634B434B2349434B634B434B234B134BE
:10052000923400342B34913492349134A0348F348B
:10053000A0348D348034A034913492349134A0347A
:100540008F34A034913480348D348D34913492348E
:10055000A034923480348D348D3492349134A0346C
:100560008F34A0348F348D3491348F34A0348D3453
:1005700000343034B934B834B93498349634A034B3
:10058000B934B834B93498349634A034B834A0347B
:10059000B6349534B834A0349834A034BB34B9346C
:1005A000BB3499349834BB34B934BB34993498345F
:1005B000B934A034B834963499349834003437348C
:1005C00099349934983494347434983498349634F3
:1005D0007234983498349634923472348F3491341F
:1005E0009234743494349534743492349934953408
:1005F000743491348F348D349434743491348F3412
:100600008D346D34003426348F34A034AF34A034AC
:10061000AF34B234A034B434A0348F34A034AF3407
:10062000A034AF34AD34A034AE348F34A034AF3402
:10063000A034AF34B234A034B434A0348F34A034F6
:10064000AF34A034AF34AD34A034AE3400341334FE
:100650008434A534603480348734A83460348034E2
:100660008434A534A034C0348734A834A034C034D2
:100670008D348B34C0348534A834A034C0348B34EA
:100680004A34A034C034AA3488348534A334853441
:1006900000343334B834A0349334BB34BA34BD346A
:1006A000BA34B634B834A0349334BB34BA34BD341D
:1006B000BA34B634BB34A0349634BF34BD34BF34FE
:1006C000BD34BA34BB34A0349834BB34BA34BB34F0
:1006D000BA34B6340034113479347934763477341A
:1006E000963477347434603479347934763497348A
:1006F00096348034743460347134713474347234A8
:100700009134723499348D348F34713491349134FE
:1007100080349134743400342B34993491349134CE
:1007200099349934A0349134913499349934913472
:10073000923491348F348F348F3498349834A03479
:100740008F348F34983498348F3491348F348D347F
:100750008D348D349634963400342034963491346C
:10076000803491349234913480349134953491347E
:10077000803492349234913490349134963491345C
:10078000803491349234913480349134953491345E
:10079000963498349934803498340034263496341E
:1007A000A0349634A0349634B934B634993496349F
:1007B00080349634A0349634A0349634BB34B634A6
:1007C0009B34963499349634A0349634A0349634BD
:1007D000B934B634993496348034943400342334A4
:1007E000913491349134913491349134A534AA34B4
:1007F000AD34B1349034903490349034903490349B
:10080000A634AA34AD34B0346F348D348A348D3488
:100810006D344A34CA34CD34D1349634003426345D
:100820008F348F34923499348034963480349634B3
:10083000943494349234963480348034B134B23465
:10084000B934B634B434B2348F348F348034AD34E8
:10085000AF34913491349434923400344034B13410
:10086000B434B1349634B434B134A034B134B43483
:10087000B134B634B634B434B134A034B134B43451
:10088000B1349634B434B134A034B134B434B13466
:10089000BB34BB34B834B434003437349234953478
:1008A000803480348034A034B5348E34923494341F
:1008B000B23495349434803480348D34913494340B
:1008C000B534943492348034A034AD348D349134C2
:1008D0009434B13492340034263468348A34AA34DF
:1008E000A834A034A8348D348834863468348F34E6
:1008F000AF34A834A034A83490348F348A34883488
:100900008F349434A834A634A034A63483348A3483
:1009100048340034403491349634993498349634C1
:100920009934963498349634923494349134803493
:100930008034A03491349634993498349634993470
:10094000963498349634913490348F34003437345C
:1009500096348D349134963498348D34913498345F
:1009600099348D349134993496349634803480346B
:100970009134923492348034803498349934983459
:10098000943496349634003430348D348D34AF340E
:10099000B234B134AF3494349434B434B634B13462
:1009A000B2348F348F34AF34B234B134AF34AD3469
:1009B000B834B634B434B234B134AF34AD340034B6
:1009C0003034B434B6349634A034B93496349634D2
:1009D0009434923494348034B434B23494348034C3
:1009E000B434B6349634A034B93496349634923450
:1009F0009634943400343034B4349234AF34B13457
:100A00009234AF34B1349234B134AF348D34B43421
:100A1000B434B234B234AF34B1349234AF34B134CC
:100A20009234B134AF348D3400342034B634803451
:100A30008034AD34B634B53480348034AD34B5341C
:100A4000B43480348034AD34B434B2348034A0341F
:100A5000AD34B234B434B534B234B63400342B349B
:100A6000963494349134B9349834B434A034B134D5
:100A7000B434B434B1349434A034B1349434A034A4
:100A80009434B434B134B9349834B43400342034A8
:100A9000B834B8349C34B834A0349A34B634803482
:100AA000803480348034A034B834B834B834B834A6
:100AB0009634B83400342634AF34B934A034AF346B
:100AC000BB34A034AF34B934A034AF34BB34A03419
:100AD000AF34AF34BE3400342034B434B2348A344A
:100AE0008C34B134AF3486348834AF34AD3485348B
:100AF00088348D3400342B34AD349234A034AD348A
:100B00009934A034B2349634B434B63492348D343B
:100B100000341034CD34CE34CF34CE34CD34003420
:100B2000103481348034813400341034D9340034AA
:100B30002000A0008B13823021009500F9143B2E79
:100B400095302000A3008530392E8930A3008530F0
:100B5000392E362EEF30A3008330392E6C30A300AF
:100B60008430392E6930A3008130392E3530A3000E
:100B70008130392E9B30A3008130392E6B30A30099
:100B80008330392E0030A3008130392E2730A30066
:100B90008330392E8C30A3008330392E0F30A300E0
:100BA0008430392EDF30A3008230392E8A30A30002
:100BB0008430392E0330A3008330392E4730A30010
:100BC0008530392EFB30A3008430392EC430A30089
:100BD0008430392E6C30A3008530392EB930A30013
:100BE0008230392E2E30A3008430392EE030A3001D
:100BF0008430392E1530A3008530392E5B30A300A8
:100C00008530392EC730A3008130392E2F30A30014
:100C10008530392EAD30A3008330392ECE30A3007D
:100C20008330392E7B30A3008530392EF130A3007C
:100C30008130392E1A30A3008230392E9230A30031
:100C40008230392EA730A3008430392E4D30A300D6
:100C50008430392E4230A3008230392E4930A3002F
:100C60008330392E6A30A3008230392E9030A300B1
:100C70008530A400462E2000200884002B3004027A
:100C80000318362E80313D3004078200230884008B
:100C9000240885000008F2007208A1000130A307B3
:100CA0000030A43D79102308840024088500120038
:100CB0000319112F23088400240885000008F2007E
:100CC0007208A2000130A3070030A43D792E403005
:100CD000722E2030722E1030722E0830722E043098
:100CE000722E0230F2007208F600962EF601F60A15
:100CF000962E2208E039F200F3017308003A031936
:100D0000822E762E7208203A0319672E603A031954
:100D1000692E203A03196B2EE03A03196D2E203A02
:100D200003196F2E603A0319712E762E7608F200A1
:100D30007208F700E12EEE30C82EE130C82ED43014
:100D4000C82EC830C82EBD30C82EB230C82EA8302C
:100D5000C82E9E30C82E9630C82E8D30C82E8530B5
:100D6000C82E7E30C82E7630C82E7030C82E69301E
:100D7000C82E6330C82E5E30C82E5930C82E54306D
:100D8000C82E4F30C82E4A30C82E4630C82E4230AA
:100D90009B000630DF2EFC30DA2EEE30DA2EE1300A
:100DA000DA2ED430DA2EC830DA2EBD30DA2EB23058
:100DB000DA2EA8309B000530DF2E9B0107309C0007
:100DC000F72E22081F39F200F3017308003A0319C5
:100DD000EA2EDD2E7208FF3E031CDD2E84001F303C
:100DE00004020318DD2E80316830040782002108D8
:100DF000F2007208A6007D3095008B161B36250088
:100E000091000C3093008B17082F20008C1C0A2FA8
:100E1000791C052F8B1325009301791020008C1865
:100E2000532EF9108430210095008B170800200004
:100E30000C188C1C172F0C1A1B2FF401F301F30A4A
:100E4000093073020318422F20000C1E242F743522
:100E5000F2007208F4000C1D302F74080138322F94
:100E60007408FE39F2007208F4001830F200F20B38
:100E7000372F00320130F2007208F3070930730295
:100E8000031C242F7408F20072082000A50008003B
:100E90006B30210099008B012500930122001D1465
:100EA000173020008C00173022008C0023008C01AA
:100EB000173021008C00843095007D30F5007508D6
:100EC0002000A700F801F910F601F701A60179103A
:100ED000A501063095008B168B1720000C1C8C1872
:100EE000722F172720000C186D2F250898256D2FBD
:020000040001F9
:02000E00C4C963
:00000001FF
